:020000020000FC
:100000000C94FD0ED0C100000000000000000000B4
:1000100000000000000000000000000000000000E0
:10002000000000002EC000000000000098C000008A
:1000300000000000000000000000000000000000C0
:10004000A1C000000000000000000000000000004F
:100050000000000002030406080C10182030406065
:1000600080000406080C10182030406080A0C000FA
:100070000003070F1F000D0D04050D050205030306
:1000800002004FB662FD0DC0552049F00994C52D00
:10009000C095089483FDC795C093B20064604FBEBD
:1000A0001895C0910401089483FDC795C093B200D0
:1000B0006B7FC0910401CF3F09F419C04FBE2B984C
:1000C0002C982D9818952B982C982D9876FD0DC06E
:1000D00064FD0BC0C5E0CA95F1F7C0915101C0FDA8
:1000E0002A9AC1FD289AC2FD299A4FBE18952092DE
:1000F000B200CC27C160C7BB6460F7CFC8CF70FF28
:10010000C6CF64FDC4CF2B9AC2CF70FFC0CF64FDB1
:10011000BECF2C9ABCCF70FFBACF64FDB8CF2D9A5A
:10012000B6CF2A9870FFB3CF64FDB1CFC1E4CA95B2
:10013000F1F72B9AACCF289870FFA9CF64FDA7CF19
:10014000C1E4CA95F1F72C9AA2CF299870FF9FCFEE
:1001500064FD9DCFC1E4CA95F1F72D9A98CF4FB6B3
:10016000C0916F00CD7FC0936F006E7FC0918400FF
:10017000CE0DD0918500DF1DD0938900C0938800FB
:100180004FBE18953FB68F7EADB3A170A2118061AE
:10019000A0E0ADBBA0916E00AE7FA0936E007894FE
:1001A000A0910801AA2341F085FD2FC0A09108016C
:1001B000AA95A093080129C040E050E085FD15C034
:1001C000A9B196FDA095A2FD4FEFA3E096FDA2E098
:1001D000A0936900AA27A160ACBB8D7FA9B196FD51
:1001E000A095A2FD5FEF451739F7A8E161FDA09347
:1001F000080185FD03C0A8E1A093080140933601E2
:100200008160442311F02092390185FD0EC0A09138
:100210000901AA2331F0A0910901AA95A09309012F
:1002200004C08061AA27A160ACBB80FF3CC0A09144
:1002300036014A2F61FF8E7F85FD1CC0A0915401BD
:10024000A430C1F4403F08F040EFA42FA295AF7056
:100250004A0F50915601533069F0A695A69550FD6E
:1002600001C0A69552FD03C0A41B4A2F03C04A0F2C
:1002700008F44FEF40930101A72FA670A1F073FD82
:1002800012C0A0911001AA0FAA0F50913E015695DD
:100290005695541708F0452F4A0F4093010118F462
:1002A000AFEFA093010140915401443009F03AC0EE
:1002B000A0910101A093030140910301A0913B0192
:1002C0004A1708F04A2FA0913D014A1708F04A2F1B
:1002D000542EA0914001AA2309F422C0542F5A1B86
:1002E00010F4A42F50E0BA2E8894AA1FAA2EA09131
:1002F0004201A095AA22A50E58F0A0914101A21595
:1003000009F0AA95AA0EA093410148F04A2D08C011
:10031000A0914101BA1608F0A395A09341014FEFB7
:1003200040930401A0910001A395A093000161F006
:10033000F894A0916E00A160A0936E0084FF02C0AB
:10034000A1E0ADBB3FBE1895A0911401A395A09369
:10035000140141E050910801552329F085FF03C0A5
:100360005A9550930801A0913601A13018F02092BF
:1003700039010DC020923A0120924301A091390128
:10038000AF5FA093390118F0AFEFA0933901F89453
:10039000A0916E00A160A0936E0084FF02C0A1E056
:1003A000ADBB3FBE18953FB640918400509185008B
:1003B0008F7EADB3A170A2118061A0E0ADBBA09112
:1003C0006E00AE7FA0936E00789481FD25C0A2E000
:1003D00096FDA3E0A09369008260A9B196FDA09567
:1003E000A2FF05C0409305015093060141C1A3E05F
:1003F00096FDA2E0A0936900AA27A160ACBB8D7F07
:1004000085FF01C028C140E0A9B196FDA095A2FDDD
:1004100022C14093360111C1A3E096FDA2E0A09352
:1004200069008D7F61FF72C0A2E096FDA3E0A093FA
:100430006900AA27A160ACBB826040933101509350
:100440003201A0902F014A19B09030015B09BB2402
:10045000A22C4C38520518F42092350149C0A091C5
:100460007401AA2359F1483C520528F4A0E1BA2EA0
:10047000AAE0AA2E23C04836A1E05A0728F4A8E033
:10048000BA2EAFE0AA2E1AC0403DA2E05A0728F4C7
:10049000A4E0BA2EAEE1AA2E11C0403AA5E05A0758
:1004A00028F4A2E0BA2EACE3AA2E08C04839A8E08E
:1004B0005A0720F4A1E0BA2EA8E7AA2EC42EA091D4
:1004C0003301CA1AD52EA0913401DA0ADD202AF4AC
:1004D000AFEFC094D094CA1ADA0A20923501A8E08E
:1004E000A210A0E0CA14DA0618F4A1E0A093350126
:1004F00040933301509334014091310150913201C6
:1005000040932F015093300142E097C0A091050124
:100510004A1BA09106015A0B94FD82C093FD80C036
:1005200092FD7CC086FF03C0D52EC42E0CC056950C
:10053000479591FD73C05695479590FD6FC0D52E98
:10054000C42ED694C79461FD19C0AC2DAC51AD2D0D
:10055000A24008F005C0DD2089F4AC2DA85C70F441
:10056000A0910701A395AA2311F0A0930701AA3037
:1005700008F471C02092360181606DC0A09107011E
:10058000AA2319F0AA95A0930701A22C50915A0111
:1005900097FD06C0A0906801533011F4A09070013F
:1005A000AAEFAA0EA22DA21DCA18DA0A4FB74170EF
:1005B000533049F4442321F087FD05C0806803C00F
:1005C00087FF01C08F77442359F0533031F4AFEFE8
:1005D000C094D094CA1ADA0A03C040E050E020C0A8
:1005E000533049F4CC0CDD1CAAE0CA1AD20818F426
:1005F000A0E0CA2ED22CAFEFCA16D20418F04FEFEB
:1006000050E00EC0A0914C01CA9E412D000C441F29
:1006100050E008F012C04FEF50E00FC056954795DC
:1006200094FF07C0552309F04FEFA42FA6954A0F5A
:10063000521D4F3F520508F04FEF40933601816045
:1006400061FF09C0AFE1A095A923AB299A2F8F7D47
:10065000BB2009F48062A8E1A093080185FF03C0D4
:10066000AAE0A093080161FD03C085FD01C08F7E53
:1006700085FD03C0A6E0A0930901F894A0916E0047
:10068000A160A0936E0084FF02C0A1E0ADBB3FBE9D
:10069000189511E00AC013E008C01AE006C01EE178
:1006A00004C014E602C018EC00C005E1BB27BA95EF
:1006B000F1F70A95D9F71A95C1F708952AE338E7B3
:1006C00009C020E33CE806C02AE234EB03C025E27F
:1006D00038EC00C0B0914D01BA9509F4089512E0CC
:1006E000BB272898BA95F1F72C9ABA95F1F72C9870
:1006F000BA95F1F7289ABA95F1F7123009F02B9ACA
:10070000123009F42D9AB0914D01BA95F1F71230DB
:1007100009F02B98123009F42D98B7E8BA95F1F743
:100720001A95F1F6022FB22FBA95F1F70A95D9F77B
:100730003A9581F628980895221B39E0001F3A95D2
:1007400009F40895221F211B18F4210F8894F6CF75
:100750000894F4CF622C722CB0E08894B395221FD9
:10076000331FE0F7379527958894912E802E020B42
:10077000130B10F4192D082D10F4889401C008945F
:10078000661C771CBA9571F7172D062D0895322D2A
:1007900011232AF43A9500951095031B130BF89436
:1007A000029F712C002D129F912C802C7894780C34
:1007B000172D921C292DB4E06B2E269517950795C1
:1007C0006A94D9F7332321F000951095031B130B7E
:1007D0000895009154010430A9F1B0913601B1504F
:1007E00008F010C0B0910101B093030120921E01E6
:1007F00020921F01209220012092210120922201AB
:100800006F7D20C0609054016062B0910101B0938F
:10081000020108E317EC20911A0130911B01369573
:100820002795B62DBA9541F036952795B62DBA95F0
:10083000BA9511F0369527950E94AA0300931E01E0
:1008400010931F01089500911E01B09102010B1B2E
:1008500010911F01120928F40038BFEF1B0740F068
:1008600009C00F37120508F405C00FE710E002C0F9
:1008700000E81FEF009323011093240108950091D5
:100880002301B09120010B0F10912401B09121019F
:100890001B1F20E03091240133230AF42A95B091E4
:1008A00022012B1F1AF4203F40F00AC02F3008F419
:1008B00007C00FEF1FEF2FE003C000E010E020EFB4
:1008C00030910301B0913B013B1718F4323030F006
:1008D00009C0B0912401BB235AF004C0B091240197
:1008E000BB2332F4009320011093210120932201B5
:1008F00008952091770100912301000F10912401A8
:10090000111F0E94C70311232AF40038BFEF1B07F1
:1009100040F009C00F37120508F405C00FE710E0DA
:1009200002C000E81FEF002352F0B0910201B01B9B
:100930000B2F18F0013008F00AC001E008C0009544
:100940000F5FB09102010B0F08F001C00FEF009391
:100950002501089520917801009121011091220133
:100960000E94C70311232AF40130BFEF1B0740F098
:1009700009C00F3F120508F405C00FEF10E002C0D8
:1009800001E01FEF112352F0B0912501B01B0B2F96
:1009900018F0013008F00AC001E008C000950F5FB0
:1009A000B09125010B0F08F001C00FEF0093030178
:1009B00008950FEF71FD1FC0B0917301BB23D9F0F3
:1009C000B0911B01BB23B9F00FEF10911B010E94E6
:1009D0009C03F894B091130172FDB5E00B9F112DAB
:1009E000002D7894112309F00FEFB0913E010B1701
:1009F00010F400913E0100933D01089500911A0109
:100A000010911B0100541140B0913D0110F4BA95B2
:100A100001C0B39511F0B0933D01089500C0089551
:100A200020915501B0917A00B6FDFACF009178007F
:100A300010917900B0917A00BF77B0937A00B091AD
:100A40004A01B395B0934A01B83060F120924A014F
:100A5000B0917201BB2321F1112329F0B0914B0118
:100A6000BF3F61F009C0B0914B010B1739F020F482
:100A7000BB2321F0BA9502C0B395E1F300913B018D
:100A8000B0934B01B03050F400ECB03038F400E8D3
:100A9000B03020F400E4B03008F400E000933B01F3
:100AA0007F7E089510913B01B0E11B0F08F41FEF0A
:100AB00010933B01B0915401B43081F000913B019F
:100AC000B0910301B01B10F400910301B0913D01FE
:100AD0000B1708F00B2F502E00930401B0914A0120
:100AE000B73009F47061089502E3F894B091790188
:100AF0000B9F012D000C001F7894B0913B010B1748
:100B000010F000913B010093010100930301502E6E
:100B10000093040100933E01089520921A01B0EF62
:100B2000B0931B010895F894009184001091850002
:100B30002091140178943091150160901601009372
:100B4000150110931601031B160971FD03C077FDF3
:100B500080C028C070901701209317012709222315
:100B600019F00FEF1FEF0EC080901801909019013F
:100B7000309318016092190100911501109116012E
:100B80000819190920911A0130911B0136952795F2
:100B9000020F131F10F40FEF1FEF00931A011093B1
:100BA0001B012BC020911A0130911B013901B4E0C7
:100BB0008B2EB2E09B2E343040F08A949A943830D9
:100BC00020F072FD02C08A949A94769467948A9475
:100BD000E1F726193709992021F0169507959A947F
:100BE000E1F7200F311F20931A0130931B0128F4E5
:100BF0003FEF30931A0130931B01323008F47068D4
:100C000071FF02C0B3E00DC0B09164010091110109
:100C1000023838F0B395003A08F0B395B63008F0D2
:100C2000B5E09B2EB4E08B2E10911B0100911A01B0
:100C300024E0169507952A95E1F70819120928F07E
:100C4000B02FB250B12FB20910F402E010E09801B9
:100C500026C020911A0130911B01390176946794C6
:100C60006694669466942619320906950695200FB7
:100C7000321D20931A0130931B01323008F07F7728
:100C800004E0369527953695279526952695201BC1
:100C900010F0223008F422E089019090640160FD98
:100CA000FECFE0902B01F0902C016160B0916F00BD
:100CB000B260B0936F00380177FD41C076946794BD
:100CC00000932B0110932C01B92DB330E1F0B0FD4E
:100CD00004C0060D171D930106C0000F111F02501E
:100CE000120922E030E0B92DB33068F020932D01D5
:100CF00030932E010093270110932801609229015F
:100D000070922A013AC000932D0110932E01209376
:100D10002701309328016092290170922A0171FF06
:100D20000DC0BFE0B0932D0120922E01B093290198
:100D300020922A01B0932B0120922C011EC06694B0
:100D400000932B01B92DB33091F0B0FD03C0060D17
:100D5000262D03C0000F025022E0B92DB33038F029
:100D600020932D01009327016092290106C0009372
:100D70002D01209327016092290100911C0102FDA1
:100D80000350013039F495FD0EC0B5E0B06CB0935E
:100D90007C000DC0023029F4B4E0B06CB0937C004C
:100DA00006C095FDF2CFB3E0B06CB0937C0000912B
:100DB0004201000F10F4BBE60B270093420160FDD7
:100DC000FECFB2E0B0930E016160B0916F00B260EF
:100DD000B0936F00B72FB67001F120911A013091D6
:100DE0001B01369527953695279571FF02C0B0E413
:100DF0003B0FF8940091840010918500020F131F9F
:100E000010938900009388006160B2E0B6BBB09196
:100E10006F00B260B0936F0078940895686020927C
:100E20001D0120E066FD20E206C0686020921D01E1
:100E300020E266FD20E001E011E077FD11C0B72F50
:100E4000B67009F0677F14E100911B01069509F463
:100E500003950F3008F00FE071FF02C004E114E1C8
:100E600060FD10C0B0911D01BB2361F071FF06C091
:100E7000B0910E01BA95B0930E0111F470625AC090
:100E80000E94E406B0917B00BF7BB0937B00B0B7BB
:100E9000B0917B00B064B0937B00B0911D01B3951D
:100EA000B0931D01B0B777FD06C0B1E071FDB3E0AE
:100EB000BA95F1F7B0B7B072B21709F030C071FF50
:100EC00005C00395011708F00A95CACF63FD05C058
:100ED0000395011708F0AFCFC3CF677FF894309127
:100EE00084006090850070901A01B0911B01770C0E
:100EF000BB1F08F4BFEF770CBB1F08F4BFEF370D23
:100F00006B1E60928900309388006160B2E0B6BBCE
:100F1000B0916F00B260B0936F0078948CCFB091B5
:100F20000D01B13008F487CF63FD85CF0A9509F034
:100F300097CF7F7D20912D0130912E01F894B2E062
:100F4000B6BB0091840010918500020F131F10930F
:100F5000890000938800E0902701F09028016160EB
:100F6000B0916F00B260B0936F007894B72FB670F5
:100F700039F0B0910D0172FFB395B0930D0109C026
:100F800075FF07C066FD05C063FD03C0BF91BF913B
:100F900097C5089500E063FF01C001E0F894109147
:100FA0001101B7E01B9F212D102D7894200F26955D
:100FB00017952695179526951795109311011837B3
:100FC00018F4B8E7B093110100911101B09112012A
:100FD0000B1720F060612B982C982D9860FDFECFA8
:100FE000E0902901F0902A016160B0916F00B26039
:100FF000B0936F000895B2E095FD0AC0F894B093E5
:101000001C0128982A9A62FF01C02D9A7894F4C096
:10101000F894B0931C012898299A62FF01C02B9A7A
:101020007894EAC0B3E082FF24C095FD11C002E0CD
:10103000F894B0931C01EBE9F0E0009351012D9876
:10104000299862FF02C02C9A01C0289A7894D4C0D3
:1010500002E0F894B0931C01EBE9F0E00093510139
:101060002B982A9862FF02C02C9A01C0289A789483
:10107000C3C095FD0BC0F894B0931C01E5E8F0E007
:101080002D9862FF01C02C9A7894B6C0F894B09362
:101090001C01E5E8F0E02B9862FF01C02C9A7894DF
:1010A000ABC0B4E095FD0AC0F894B0931C012A9837
:1010B000299A62FF01C02C9A78949EC0F894B0934C
:1010C0001C0129982A9A62FF01C02C9A789494C036
:1010D000B5E082FF24C095FD11C001E0F894B09303
:1010E0001C01E1E9F0E0009351012C98289862FF7F
:1010F00002C02B9A01C02A9A78947EC004E0F8942A
:10110000B0931C01E5EAF0E0009351012C98289877
:1011100062FF02C02D9A01C0299A78946DC095FD96
:101120000BC0F894B0931C01EFE7F0E02C9862FF3D
:1011300001C02B9A789460C0F894B0931C01EBE83E
:10114000F0E02C9862FF01C02D9A789455C0B6E06B
:1011500095FD0AC0F894B0931C012998289A62FF63
:1011600001C02B9A789448C0F894B0931C012A9837
:10117000289A62FF01C02D9A78943EC0B1E082FFA8
:1011800024C095FD11C004E0F894B0931C01E5EA79
:10119000F0E0009351012B982A9862FF02C02D9A2B
:1011A00001C0299A789428C001E0F894B0931C01FA
:1011B000E1E9F0E0009351012D98299862FF02C007
:1011C0002B9A01C02A9A789417C095FD0BC0F89409
:1011D000B0931C01EBE8F0E02B9862FF01C02D9A60
:1011E00078940AC0F894B0931C01EFE7F0E02D98D2
:1011F00062FF01C02B9A78946F7E08952EE730E04D
:10120000F901209251012B982C982D982A98289812
:1012100029986B7F0895A2E5B1E009E00D9309E0FC
:101220000D9304E00D930FEF0D9303E00D930FEF7B
:101230000D930BE00D9301E00D9301E00D9301E0A0
:101240000D93AEE5B1E001E00D930FEF0D930D931B
:101250000D930D930D9303E00D930FEF0D930FEF8F
:101260000D930D9305E20D9300ED0D9308E20D93A0
:1012700000E50D9304E00D930FEF0D9302E00D9345
:1012800000E00D930AE70D930FEF0D9300E00D932F
:1012900001E00D9300E00D9303E00D9300E00D934A
:1012A0000895209159018B7FB0915A01B33019F004
:1012B0009F7DB1FD90629F7BB0915B01B1FD906419
:1012C000223011F0886001C0877F08950A95E00FF1
:1012D000F21DB4910895E4E5F0E0009152010E94FE
:1012E0006609B0937701E4E5F0E0009153010E94B4
:1012F0006609B0937801E2E6F0E0009158010E949F
:101300006609B093790100915801023008F402E0B7
:1013100000931301B0916E010FEFB23009F400EAAF
:10132000B33009F402E800931201E0E7F0E0009125
:1013300075010E946609B0934001089508952091B7
:10134000680130916901B0915A01B33009F43E50FF
:1013500097FF02C020E03FEFB32FB21B6B2EB258B5
:1013600010F4B2E86B2E00E00395609EB12DBD57DE
:10137000D8F300934C01089590680E949F090E9441
:101380004F030E944F0320E030E0B0E16B2E0E943B
:101390004B03B09136012B0F321D6A94C1F7B4E0B4
:1013A00036952795BA95E1F7822E9F770E949F097F
:1013B0000895F894E3E0F0E0B9E0B7BFB491B078F5
:1013C000C1F3F894A895B4B7B070B4BFB091600001
:1013D000B861B0936000B0E0B0936000B4E0BEBF0D
:1013E000BFEFBDBF0E94FE08B0E0B5B9BFE3B4B91E
:1013F000B0E0B8B9B0E0B7B9B0E0BBB9B0E0BAB9E5
:101400002224A0E0B0E02D92AA31E9F7A0E0B1E0FB
:101410000FEF2D920A95E9F7B1E0B09342010E94D7
:101420000B090E94A30DB0E0B06CB0937C00B091AA
:101430007A00B460B068B0937A0000916A010093BA
:101440004D01B1E0B0930A01F8940E9453030E9449
:101450005E030E944F030E9461030E944F030E949B
:1014600064030E944F03F8940AEF1AEFA9B196FDA6
:10147000A095A2FF1FC01A95C9F70A95B1F7E0E041
:10148000FCE3B591B43E39F4B591B03E21F4B59189
:10149000BF3F09F40CC0E0E0F395F395B591B83F78
:1014A00049F4B591B43931F4B591BA3A19F4EE274B
:1014B000F69509940E9451090E946B090E949E09A9
:1014C0000E949F0900916A0100934D010E94FE084D
:1014D000B2E0B5BDB2E0B0938100B2E0B093B1002C
:1014E000B1E0B5BBB0936E00B2E0B6BBB0936F0095
:1014F000B1E0B7BBB0937000B0917B00BF7BB093FD
:101500007B00B0B7B0917B00B064B0937B000E94C9
:10151000490378940E940E0520921001B3E096FDD5
:10152000B2E0B0936900B1E0BDBBBB27B160BCBB0A
:101530008D7F0E945303626033E02CE0B09135014F
:10154000BB2321F42CE03A9509F48DCF0E944F0380
:1015500080FF89CF8E7FB0913601B23070F3B92F02
:10156000BF710091380100933701B0933801B01773
:1015700021F72A9519F76D7FB3E096FDB2E0B0939D
:101580006900BB27B160BCBB8D7FB0917401BB23E8
:1015900021F48062B92FB0709B2F8F7B20920701BE
:1015A0000E94510385FF05C0B0910701BA3008F0D1
:1015B00080640E944B0302E085FF01C000E0B0910F
:1015C0003601B017B0F3F8940E945E030E945E03E8
:1015D0000E945E0378940E94530320922601B091EA
:1015E0005A01B33009F499C00E944B03B0915E01D7
:1015F000B13008F492C0B0910A01B13008F48DC046
:1016000085FD1EC0B0913601BF3F08F486C0F89436
:101610000E94670378940E945103B0913601B13063
:10162000B0F7F8940E945E030E944D030E945E038F
:1016300078940E945103B0913601BF3F90F375C377
:10164000B3E09B2E9068F8940E949F0978940E94C2
:101650005103F8949F770E949F0980903601B091C2
:101660003601BF37789408F460C00E944903F894AB
:101670000E94670378949A9429F70E94BC09B82DB8
:10168000B09369010E945303F8940E94460E789427
:10169000BAE09B2E9068F8940E949F0978940E946B
:1016A0005103F8949F770E949F0980903601B09172
:1016B0003601BF37789460F70E944903F8940E947E
:1016C0005E030E944D030E945E0378949A9411F782
:1016D0000E94BC09B82DBB5FB09368010B2F10911D
:1016E0006901125810F0100B20F4B2E80B0F0093B0
:1016F00069010E945303F8940E94D60D0E94630E64
:1017000078940E945103F8940E949F097894B091B4
:101710003601BF3F08F474CF08C300913601B09181
:1017200026010B1710F0009326010E94510301E0DF
:10173000B0915A01B35009F405E0B0913601B017E9
:1017400008F04DCFF8940E9467030E9467030E943F
:10175000670378940E94530320920A0120920B01A0
:1017600020920C01B0910B01B395B0930B01BF3FD8
:1017700091F5B0910C01B395B0930C01B0916C014F
:1017800009E1BA9559F002E3BA9541F00DE7BA952F
:1017900029F00AEFBA9511F020920C01B0910C01DA
:1017A000B017C8F00E94FE080E944903B0910C01D6
:1017B000BA95B0930C0120920B01B0916B01B093DC
:1017C0004D01F8940E9467037894B0916A01B09338
:1017D0004D010E9451030E944D03B0910801BB23AB
:1017E00019F485FF01C03FCE01E085FD01C006E090
:1017F000B0913601B01708F4B5CFB0915A01B3508B
:1018000011F00E945103B0910801BB2309F42BCEC3
:10181000F8940E94FE082092010120920201209279
:101820000301522C20920401209241017894B0913E
:101830005701BB0FB0933F0120921E0120921F0160
:1018400020922001209221012092220120924A011F
:1018500060E070E020921101B8E0B0934A0170613D
:101860000E944903B0E074FDB0E0B06CB0937C001E
:10187000B0917A00B068B064B0937A00B0917A0009
:10188000B6FDFCCF0091780010917900B0917A00FC
:10189000BF77B0937A00112309F00FEF00934B014B
:1018A0000E941005B8E0B0934A0170610E9451098E
:1018B000F894BFEFB0933B010E947405B091010111
:1018C000B0933B01B0933C01B0933D017894B1E0FB
:1018D000B0930101B09303015B2EB0930401B09368
:1018E0004401B0913A01B0934301B0915A01B33031
:1018F00019F49F7D87FD90627160726020920D01E6
:101900000E94A7080E94BE080E948D050E949305B0
:101910000E948D050E9493050E948D050E94150767
:101920000E94E9030E94CA070E94FB070E949305D8
:101930000E940E0765FD0E94230477FF0E94D904D0
:1019400077FD0E94FE040E94CA070E9412080E94AE
:1019500093050E94150765FD0E943F040E94CA0777
:101960000E9451080E9493050E940E0765FD0E9487
:1019700079040E94CA070E9468080E9493050E9489
:10198000150765FD0E94AA040E94CA070E94A708C5
:101990000E9493050E940E07B0E074FDB0E0B06CA9
:1019A000B0937C00B0917A00B068B064B0937A00D4
:1019B0000E94CA070E94BE080E9493050E9410055B
:1019C00071FF24C0B0913E01B0933B01B0933C0144
:1019D000B0913A01B0934301B1E0B093440118E1F2
:1019E0002CE0B0910D01B11758F07D7F7460209309
:1019F0000F01B0913E01B0933B01B0933D0106C091
:101A0000B0913601B13008F089CF64C072FF15C0C3
:101A100066FD13C0B0910F01BA9519F47B7F786011
:101A20007DCFB0930F01B0913601B13008F076CF81
:101A3000B0915A01B33009F04DC020921001B0911D
:101A400039010AEF10917601112309F003E0B01774
:101A500008F040C085FF04C0B0910801BB23D1F15C
:101A6000B0915A01B33081F495FD03C087FD04C0E5
:101A70000BC087FF01C008C066FD06C06064B0915E
:101A80003E01B0933B0170CF00EF66FF05C0B091FF
:101A90003E01B0933B0100E2B0911B01B01708F486
:101AA0003DCF66FF17C06F7B9F7D87FD906274609E
:101AB000B2E1B0930F01B0913E01B0933B012ECF44
:101AC000B0911001B395B0931001B0913601BB23D2
:101AD00009F002C020921001F8940E94FE08809044
:101AE0005901B2E0B09359010E9451098092590105
:101AF000209201012092020120920301522C209297
:101B0000040120923F0160E070E078940E9451034C
:101B10000E94FE0800917601002319F02B9A2C9A5E
:101B20002D9AB0E0B06CB0937C00B0917A00B460B4
:101B3000B068B0937A0085FF05C0B0911001B43051
:101B400008F091CC0BCEEDE0F0E00E94CF0D053512
:101B500009F01EC0EEE0F0E00E94CF0D0A3A09F055
:101B600017C03AE0A2E5B1E0E3E0F0E00E94CF0D5B
:101B70000D9331963A95D1F739E1AEE5B1E0EFE05A
:101B8000F0E00E94CF0D0D9331963A95D1F704C045
:101B90000E940B090E94D60DE8E2F0E00895F99941
:101BA000FECFE1BDF2BDF89A00B508950E94F90D8F
:101BB0003AE0A2E5B1E0E3E0F0E00D910E94F10D22
:101BC00031963A95D1F739E1AEE5B1E0EFE0F0E0DA
:101BD0000D910E94F10D31963A95D1F70E94040EB5
:101BE0000895F999FECF00BDE1BDF2BDFA9AF99AC8
:101BF0000895EDE0F0E00FEF0E94F10DEEE0F0E06F
:101C00000FEF0E94F10D0895EDE0F0E005E50E9470
:101C1000F10DEEE0F0E00AEA0E94F10D0895309136
:101C20004E0100914F01313011F4009352013230D6
:101C300011F400935301333011F400935401343004
:101C400011F400935601353011F4009358013630E9
:101C500011F400936401373011F4009359013830C6
:101C600011F400937501393011F400936E013A308C
:101C700011F400935A013B3011F400935B01089575
:101C800025E00E9453032A95E1F708950E945E0320
:101C90000E9461030E9464030E9467030E944D0337
:101CA0000E945E030E9461030E9464030E94670316
:101CB0000E944D030E945E030E9461030E94640320
:101CC0000E94670308950E9467030E9464030E94B4
:101CD00061030E945E030E944D030E9467030E94FD
:101CE00064030E9461030E945E030E944D030E94F0
:101CF00067030E9464030E9461030E945E030895CB
:101D000080904E0190904F010E945E030E945E03FE
:101D10000E945E030E944D038A94B1F70E946703FC
:101D20000E944D039A94D1F70895F8940E94460EAC
:101D300078940E94400E0E94400EB1E0B0934E0194
:101D4000B1E0B0934F0120925001F8940E94800EB0
:101D50007894B5E06B2E709036010E945303B091D9
:101D600036017B16C1F7B13018F0BF3F70F10CC0DF
:101D70000E940F0EF8940E94D60D0E94460EB8E005
:101D8000B09360000E94400E6A9429F7B091500110
:101D9000B395B0935001B33008F4D7CF0E94400EF2
:101DA000B0914F01B395B0934F01F894B0914E01AB
:101DB000BA95E6E7F0E0EB0FF21D049178940395F5
:101DC000B0914F01B01708F4BECF0E94400E0E94A0
:101DD000400EB0914E01B395B0934E01B0914E01BB
:101DE000BC3008F4ADCF0E940B09F8940E94D60DC8
:0C1DF000B8E0B09360000E94400EDBCA17
:00000001FF
